:1000BD0001020304050607080901010102020203FA
:0200CD0003032B
:1000030078087C007D007BFF7A0079BD7E007F0944
:100013001201AB78117C007D007BFF7A0079C67EEC
:10002300007F091201ABE4F52F753000753101E44F
:10003300F52CE4F52DE4F532F533F52EE52E75F0C8
:1000430003A42411252DF8E6FD3395E0FCE52C757A
:10005300F003A42408252EF8E6FF3395E0FE1201F1
:10006300D4EF2533F533EE3532F532052EE52EB4D4
:1000730003CAE52C75F006A4241AF8E52D25E0281B
:10008300F8A63208A633052DE52DB403A8052CE503
:100093002CB4039E0531E53170020530E53164E887
:1000A3007004E53064037087852F90052FE52F6476
:0A00B3000A600302002C0200032281
:030000000200CF2C
:0C00CF00787FE4F6D8FD75813302000351
:1000DB00E709F608DFFA8046E709F208DFFA803E07
:1000EB0088828C83E709F0A3DFFA8032E309F608F4
:1000FB00DFFA8078E309F208DFFA807088828C835C
:10010B00E309F0A3DFFA806489828A83E0A3F6080F
:10011B00DFFA805889828A83E0A3F208DFFA804CE9
:10012B0080D280FA80C680D4806980F280338010C0
:10013B0080A680EA809A80A880DA80E280CA803329
:10014B0089828A83ECFAE493A3C8C582C8CCC583A1
:10015B00CCF0A3C8C582C8CCC583CCDFE9DEE78071
:10016B000D89828A83E493A3F608DFF9ECFAA9F0F0
:10017B00EDFB2289828A83ECFAE0A3C8C582C8CC46
:10018B00C583CCF0A3C8C582C8CCC583CCDFEADE5F
:10019B00E880DB89828A83E493A3F208DFF980CCC1
:1001AB0088F0ED2402B4040050C2F582EB2402B4B3
:1001BB00040050B823234582F582EF4E60AEEF600A
:0901CB00010EE5822390012B7363
:1001D400EFF88DF0A4FFEDC5F0CEA42EFEEC88F070
:0401E400A42EFE2225
:00000001FF
